:1000000012C0189518951895189518951895189563
:100010001895189518951895189518951895189578
:100020001895189518958FED8DBFC0ECE0EC4E2E0D
:10003000DD275D2EEEE7F0E0A0E6B0E088278D93A7
:100040003197E9F77ED266248FEF81BB80E082BBD7
:1000500084E690E0EAD28DE0BCD259D28FE711E17C
:1000600065D2EEE1F7E04BD281E08093620000912F
:1000700062000F3010F009F00BC088E1AAD28AEFBD
:1000800090E0D3D2A2E68C918F5F8C9308F4EFCFEF
:10009000E1E0F0E04DD23BD238D2EEE2F7E02FD2F1
:1000A00084EF91E0C2D2E4E3F7E029D284EF91E05B
:1000B000BCD2EAE3F7E023D288EC90E0B6D2EEE3DC
:1000C000F7E01DD288EC90E0B0D2E0E4F7E017D280
:1000D00088EC90E0AAD2E2E4F7E011D288EC90E05C
:1000E000A4D2E6E4F7E00BD288EC90E09ED2E8E4FC
:1000F000F7E005D284EF91E098D28FEB1DE016D2A5
:10010000EAE4F7E0FCD188EC90E08FD2EAE4F7E093
:10011000F6D188EC90E089D2EAE4F7E0F0D188ECFF
:1001200090E083D2EAE4F7E0EAD184EF91E07DD277
:100130008FEB1DE0FBD1E8E4F7E0E1D188EC90E043
:1001400074D2ECE4F7E0DBD188EC90E06ED2EEE420
:10015000F7E0D5D188EC90E068D2E0E5F7E0CFD1C8
:1001600084EF91E062D281E08093620000916200AE
:10017000003110F009F00BC08CE12BD28AEF90E037
:1001800054D2A2E68C918F5F8C9308F4EFCF8CE071
:1001900020D280E08093620080E080936300A1E63B
:1001A0008C918F5F8C93B3D1E2E5F7E0A8D188EC16
:1001B00090E03BD2E8E5F7E0A2D188EC90E035D2C0
:1001C000EAE5F7E09CD188EC90E02FD2ECE4F7E090
:1001D00096D188EC90E029D2ECE5F7E090D188EC5C
:1001E00090E023D2EEE5F7E08AD188EC90E01DD2D2
:1001F000E0E5F7E084D188EC90E017D2E8E4F7E09E
:100200007ED188EC90E011D2ECE4F7E078D1E2E026
:10021000F0E08ED17AD100916100013009F002C086
:1002200038D1E2C000916100023009F024C0E2E65A
:10023000F7E065D1F2D088EC90E0F7D1E8E6F7E09E
:100240005ED1EBD088EC90E0F0D1EAE6F7E057D150
:10025000E4D088EC90E0E9D1ECE6F7E050D1DDD0D5
:1002600088EC90E0E2D1EEE6F7E049D1D6D0E1E0CB
:10027000F0E05ED15BC000916100033009F001C085
:10028000D5C000916100043009F03BC040D188EC3A
:1002900090E0CBD1E0E7F7E032D137D184EF91E0C5
:1002A000C4D1E0E8F7E02BD1B8D088EC90E0BDD124
:1002B000E6E8F7E024D1B1D088EC90E0B6D1E8E8E8
:1002C000F7E01DD1AAD088EC90E0AFD1EEE6F7E0E0
:1002D00016D1A3D084EF91E0A8D175D0E1E0F0E091
:1002E00027D115D188EC90E0A0D1EAE8F7E007D15A
:1002F0000CD184EF91E099D1CCD0E1E0F0E018D1BD
:100300000CC000916100053009F003C080E08093CB
:100310006100E1E0F0E00CD19BCEF9D0EAE9F7E032
:10032000EED051D0E2E0F0E003D133CF939AEFD09A
:10033000EAEAF7E0E4D084EF91E077D1E8D084EF07
:1003400091E073D1EAEAF7E0DAD084EF91E06DD181
:10035000DED084EF91E069D1EAEAF7E0D0D093985B
:10036000E1E0F0E0E5D0D1D0E8EBF7E0C8D08AE0FA
:10037000809360004091600001E0041710F009F0E4
:1003800021C08FEB19E0D2D0009160000A3008F054
:1003900003C0EEE6F7E0B3D0A8EAB0E0E0E6F0E0B4
:1003A00074D1A5D08FEB1BE0C1D0E2ECF7E0A7D071
:1003B000E1E0F0E0BDD0809160008150809360006A
:1003C00008F0D8CFE6CE84E690E02FD1939A88EC5F
:1003D00090E02BD1939888EC90E027D1939A88EC09
:1003E00090E023D19398089584E190E01ED18FD0BE
:1003F000EAE9F7E084D0E7DF88D0E8ECF7E07FD0E7
:100400008CE291E012D1949AE2E0F0E091D09498DD
:100410007ED084E690E009D13ECE939A84E690E0C7
:1004200004D1939884E690E000D1089570D0CBDF9A
:100430008FE0CFD06CD0E6EDF7E061D084EF91E0B3
:10044000F4D0E0EEF7E05BD084EF91E0EED05DD049
:10045000E6EEF7E054D084EF91E0E7D0E0E8F7E093
:100460004ED084EF91E0E1D0E6E8F7E048D084EFA9
:1004700091E0DBD0E8E8F7E042D084EF91E0D5D01E
:10048000EEE6F7E03CD0E1E0F0E052D08CE0A1D025
:1004900080CEE2E6F7E033D0C0DF88EC90E0C5D054
:1004A000E6E8F7E02CD0B9DF88EC90E0BED0E8E6D3
:1004B000F7E025D0B2DF88EC90E0B7D0E8E6F7E0CF
:1004C0001ED0ABDF88EC90E0B0D0ECE6F7E017D0C0
:1004D000A4DF88EC90E0A9D0ECE6F7E010D09DDF37
:1004E00088EC90E0A2D0E1E0F0E022D00895A8EA04
:1004F000B0E08D91882311F066D0FBCF0895A4D091
:10050000802D11F060D0FBCF089580EC62C081E0B7
:1005100060D014D080E85DC08FE7213039F08FEBD8
:10052000223021F08FE8233009F08FEC810F51C089
:1005300088EE93E07AD03197D9F7089583E0992730
:1005400074C08AEF90E071D0BB9ABA9AB99AB89AFF
:100550008E9A8D9A959885E090E067D09698C3988A
:10056000C298C19AC09A969AEF93FF93E4ECF0E098
:1005700050D0FF91EF91969855D0969AEF93FF93B4
:10058000E4ECF0E046D0FF91EF9196984BD0969A2C
:10059000EF93FF93E4ECF0E03CD0FF91EF9196985D
:1005A00041D0C098969AEF93FF93E4ECF0E031D0FD
:1005B000FF91EF91969836D088E20BD08EE009D06B
:1005C00086E007D00895959A829505D004D02AD068
:1005D00008959598F9CF859510F4C09A01C0C098F8
:1005E000859510F4C19A01C0C198859510F4C29AFE
:1005F00001C0C298859510F4C39A01C0C398969A19
:10060000EF93FF93E4ECF0E004D0FF91EF91969824
:1006100008953197F1F70895689462F80895E89481
:1006200062F8089581E090E000C0EF93FF93EE2719
:10063000E82BE92B31F0E0EDF7E03197F1F7019786
:10064000D1F7FF91EF910895C89531960020089554
:10065000000F111F221F331F08950095109520953C
:1006600030950F5F1F4F2F4F3F4F0895019110811D
:100670000EC001911191219130810BC00191108127
:1006800017FF05C03FEF2FEF04C00081112722277D
:10069000332737FF03C0E1DF8DE28D93CF93DF93E4
:1006A000CF92DF92EF92AA24BB24CC24DD24EE2447
:1006B00040E2CAE0DD2755E093E38881890F87FD9A
:1006C0009F7083FD907F891B89935A95A9F7C0DF9E
:1006D000AA1CBB1CCC1CDD1CEE1C4A9551F7E894EF
:1006E000EFE0FF2782910ED0EB30E0F71EF0689428
:1006F0008A2D0CD088278D93EF90DF90CF90DF91DB
:10070000CF910895982F829501D0892F8F70805DA9
:1007100026F0803309F4089568948D93089557570F
:10072000572E4156522E344D472E434F4D00436FA6
:10073000646500004C6F636B0000204100005600B0
:100740005200206C0000630064002D0065006D0005
:100750006F002020204500006E00740072002063AE
:100760000000202020320000340036003800300025
:1007700020456E746572206F6C6420636F64650041
:100780002020203100003200330020456E74657255
:10079000206E657720636F64650020436F64652079
:1007A00061636365707465640000202020436F649A
:1007B000652077726F6E67002020576169743A2058
:1007C000000020736563000020202020556E6C6FB0
:1007D000636B656400002020496E697469616C0078
:0E07E00020636F6465002020202020697300D4
:00000001FF
